:100000006AC0000084C0000082C0000080C0000000
:100010007EC000007CC000007AC0000078C00000F4
:1000200076C0000074C0000072C0000070C0000004
:100030006EC000006CC000006AC00000B1C30000C8
:1000400066C0000064C0000062C0000060C0000024
:100050005EC000005CC000005AC0000058C0000034
:1000600056C0000054C0000052C0000050C0000044
:100070004EC000004CC000004AC000000800000054
:10008000BE922449123EABAAAA2ABECDCCCC4C3E8D
:1000900000000080BEABAAAAAA3E00000000BF007C
:1000A0000000803F0000000000084178D3BB438778
:1000B000D1133D190E3CC3BD4282AD2B3E68EC828C
:1000C00076BED98FE1A93E4C80EFFFBE01C4FF7F11
:1000D0003F000000000011241FBECFEFCDBFDFE3C3
:1000E000DEBF8091400080934000811105C098EDF3
:1000F00021E094BF209341008CBB2AE3A0E0B8E349
:1001000001C01D92AA30B207E1F779D380C778CF3A
:100110002F923F924F925F926F927F928F929F9217
:10012000AF92BF92CF92DF92EF92FF920F931F9305
:10013000CF93DF93CDB7DEB7C05FD140CDBFDEBF79
:100140002AE038E3CD51DE4F28833983C35ED140A6
:10015000C12CD12C7601CD51DE4FE881F981C35EEF
:10016000D140A191B191CD51DE4FE883F983C35EB7
:10017000D1409D0105D7C60ED71EE81EF91EEA50D4
:10018000FA4349F7C11434E0D306E104F1040CF456
:10019000BEC180EE91E0FE013196DF019C011D920F
:1001A00021503040E1F7AE014B5A5F4FCF51DE4F47
:1001B00048835983C15ED140C151DE4F4883598382
:1001C000CF5ED1404BEE842E912CA12CB12C00E0BF
:1001D00010E0C401880F991FCD51DE4FA881B9816D
:1001E000C35ED140A81BB90BC551DE4FA883B983AC
:1001F000CB5ED140EAE0F8E3C351DE4FE883F983F8
:10020000CD5ED140312C212CC12CD12C7601C9518D
:10021000DE4F188219821A821B82C75ED140412CA0
:10022000512C32012814390408F044C0C351DE4F68
:10023000E881F981CD5ED14041915191C351DE4FAA
:10024000E883F983CD5ED140C551DE4FA881B981E5
:10025000CB5ED140ED91FD91C551DE4FA883B983AE
:10026000CB5ED1409A01DF018BD6460E571E681E29
:10027000791EDA0185D6C951DE4F288139814A813C
:100280005B81C75ED140260F371F481F591FC951D8
:10029000DE4F288339834A835B83C75ED1409F0149
:1002A000DF016ED6C60ED71EE81EF91E3FEF231AD9
:1002B000330AB8CFC951DE4F88819981AA81BB81A9
:1002C000C75ED140C80ED91EEA1EFB1EC114D10460
:1002D000E104F10409F404C1C301B201A6D49B01F5
:1002E000AC01D1D32B013C01C701B6019ED49B01C7
:1002F000AC01C301B2012FD46B017C01C151DE4FAF
:10030000A881B981CF5ED140CD92DD92ED92FD9270
:10031000C151DE4FA883B983CF5ED1409501A801BA
:10032000C701B60132D5181614F456018701B1E0A1
:100330008B1A9108E8E88E16910409F04ACF2DEC4B
:100340003CEC4CE45FE3B501C80101D487FDDFC09C
:100350002BE734E14EE65FE3B501C8015FD5CD512F
:10036000DE4F688379838A839B83C35ED14026E115
:10037000222E312CCF51DE4FA881B981C15ED140F0
:100380001496CD90DD90ED90FC90179781010F5F52
:100390001F4FCD51DE4F288139814A815B81C35E79
:1003A000D140C701B601D3D387FD9EC0CF51DE4FE8
:1003B000E881F981C15ED14080809180A280B380C4
:1003C000A7019601C501B401E0D487FF8DC0CF51CC
:1003D000DE4FA881B981C15ED14018964D905D90E5
:1003E0006D907C901B97A3019201C701B601AFD31A
:1003F00087FD7AC0A7019601C701B60144D39B01CE
:10040000AC01C501B4013ED3A30192013CD36B0101
:100410007C019F772DEB37E346E855E3B6D41816F9
:100420000CF079C0A3019201C501B4012BD320E0E7
:1004300030E040E05FE3F2D4A70196018CD36B017A
:100440007C0120E030E040E05FE39FD418160CF41C
:1004500066C020E030E040E05FEBC701B60177D333
:1004600087FF05C0C12CD12CE12C9FEBF92EB101E7
:1004700090E080E0D8D3A701960105D39B01AC01A1
:1004800060E070E08AEF95E466D36B017C0120E0C8
:1004900030E04CE852E479D487FD39C020E030E008
:1004A00044EB53E4C701B60152D3181684F1C701D7
:1004B000B601C051DE4FCDBFDEBFDF91CF911F919E
:1004C0000F91FF90EF90DF90CF90BF90AF909F90F3
:1004D0008F907F906F905F904F903F902F900895F6
:1004E000C12CD12C76010ACFCF51DE4F2881398122
:1004F000C15ED1402C5F3F4FCF51DE4F28833983FF
:10050000C15ED14018010737110509F033CFC12C66
:10051000D12C7601CCCFC12CD12C7601A8CFC12C07
:10052000D12CE12C8FE3F82EA2CFCF92DF92EF9265
:10053000FF929FB7F89488E08093840A80918E0A96
:1005400081FFFCCF80918D0AE091A20AF091A30A6D
:10055000C0900038D0900138E0900238F090033815
:100560009FBF80FF08C0E730F10528F48FEFC81A5D
:10057000D80AE80AF80A9F0136952795CF01820F1D
:10058000911DE22FE695E695322F32953F70E31BE1
:10059000FF0B27FD3196E80FF91FA0E3B3E0A70199
:1005A000960109D5F694E794D794C794C60ED71E42
:1005B000E81EF91EC701B6016E0F7F1F811D911D38
:1005C000FF90EF90DF90CF900895CF92DF92EF925F
:1005D000FF92CF93DF936B017C01A7DFEB01A5DFD7
:1005E0006C1B7D0B683E7340A0F0C114D104E10484
:1005F000F10439F4DF91CF91FF90EF90DF90CF902D
:10060000089581E0C81AD108E108F108C851DC4F0B
:10061000E6CFC114D104E104F10409F7EBCF8091D6
:10062000280481700895CF93DF93823108F047C08A
:1006300090E0EC01C159DF4628812F3F09F43FC00B
:10064000AC01435A5F46DA01EC91B0E2EB9FF00156
:100650001124FC5F611136C0268330812323A1F46D
:100660009C01255B3F46D9012C91309769F12830D8
:1006700058F57096E20FF11D3FB7F8942081611193
:1006800026C0277F20833FBF875C9F46FC01908167
:100690009923A9F08881903409F1983FE1F09031D5
:1006A00071F4DA019C919130A1F4853010F0880F3B
:1006B00082959091010A809589238093010ADF91A8
:1006C000CF9108952583C9CFF0E0E0E0D5CF286031
:1006D000D9CF880FEECF1092A006F1CF823019F15A
:1006E00080E49091920A982351F34FB7F894909137
:1006F000800A9E7F9093800A2091920A90E08095D4
:10070000909530E08223932328ED24BF8093920AB2
:1007100080918E0A80FFFCCF8091800A8160809357
:10072000800A4FBFCCCF80E8DCCFCF93DF93C3E309
:10073000D0E960E0899177DF80E9C933D807C9F74C
:1007400060E086E070DF60E088E06DDF60E087E019
:10075000DF91CF9168CF8231F0F490E0FC01E15954
:10076000FF4620812F3FB9F0FC01E35AFF46E081AC
:1007700030E2E39FF0011124FC5F60FF0DC0218394
:10078000855B9F46DC018C91E80FF11D808961FF3C
:1007900005C08860808B08952283F2CF877FFACFCF
:1007A0008F9381E080938D0A8FB78F93EF93FF93A0
:1007B000E0E0F8E39F9368948FEF0DC0E8948481A4
:1007C0009581805D9C4F84839583885E934080F003
:1007D000848395838FEF9081981B919390819F4F95
:1007E000919390819F4F919390819F4F919336F376
:1007F0009F91FF91EF918F918FBF8F911895CF931C
:10080000DF93CDB7DEB72B97CDBFDEBF81E098ED8C
:1008100094BF80936100E0E0F6E092E592839DE072
:10082000958390E293838083109202028093030A5F
:100830009EEF9093260A9093270A9BE09093000ADC
:10084000E0E8FAE02DEF31E026A737A7118290E823
:100850009283848781E180837894809100068B7FE6
:100860008093000660E08FE076DF62E089E073DF6E
:1008700003E310E961E0F80181918F016CDFF0E999
:1008800009331F07B9F761E086E065DF61E088E0C2
:1008900062DF61E087E05FDF48DF1E018AE0280E4B
:1008A000311CBDDE811128C089E0E2E1F0E9DE0102
:1008B000119601900D928A95E1F737DF8E010F5F57
:1008C0001F4FF801F1908F0161E08F2DACDE66E9DA
:1008D00070E080E090E079DE60E08F2DA4DE02150C
:1008E000130579F79CDE882349F31FDF64E670E087
:1008F00080E090E06ADED5CF18DE2B013C010AE0F3
:1009000018E35801C12CD12C76010FDE641975094A
:100910008609970997FDF9CF80910006882309F48D
:10092000A0C0F2E0F093060681E080930806809173
:100930000B0680FFFCCF8091100690911106F50107
:10094000819391935F01092E000CAA0BBB0BC80E7B
:10095000D91EEA1EFB1EFDE74F0E511C611C711CC7
:100960008AE0A8168AE3B80681F6C701B60120E03E
:1009700031E040E050E0E8D2F801819191918F019F
:100980003297821B930B80839183FAE30A301F070F
:1009900099F7BEDB4B015C01C8DE20E030E0A90125
:1009A000C501B401D4D018160CF07BCF8BE190E9CF
:1009B0008A879B8700E0712C90E5692E23EC522EEC
:1009C00037E4432E10E0EA85FB8521913191419176
:1009D0005191EA87FB87C501B401BDD0DFD12DE776
:1009E00037E648ED54E41AD26B017C01E894F7F83D
:1009F000A7019601672D762D852D942DC6D1181649
:100A00002CF47C2C6D2C5E2C4F2C012F1F5F16308C
:100A1000D1F610E0F801ED5CFF4661E0808103DE75
:100A2000000F111F000F111FF801E55EFF46208126
:100A3000318142815381C501B4018DD0AFD12DE701
:100A400037E648ED54E4EAD16B017C0120E030E068
:100A500040E850EC7CD087FF07C061E086E0E3DD32
:100A600020CF89EF92E86BCF20E030E040E850E4FF
:100A7000C701B6018AD161E0181614F487E0EFCF00
:100A800088E0EDCF5058BB27AA270ED044C135D1FE
:100A900030F03AD120F031F49F3F11F41EF42AC116
:100AA0000EF4E095E7FB20C1E92F46D180F3BA1799
:100AB000620773078407950718F071F49EF55EC10D
:100AC0000EF4E0950B2EBA2FA02D0B01B901900169
:100AD0000C01CA01A0011124FF27591B99F0593FAD
:100AE00050F4503E68F11A16F040A22F232F342FF5
:100AF0004427585FF3CF469537952795A795F04043
:100B00005395C9F77EF41F16BA0B620B730B840B57
:100B1000BAF09150A1F0FF0FBB1F661F771F881F0F
:100B2000C2F70EC0BA0F621F731F841F48F4879567
:100B300077956795B795F7959E3F08F0B3CF939556
:100B4000880F08F09927EE0F979587950895A8D0FC
:100B500008F481E008950CD0DEC0D6D040F0CDD0AE
:100B600030F021F45F3F19F0BFC0511108C1C2C07D
:100B7000E3D098F39923C9F35523B1F3951B550B93
:100B8000BB27AA2762177307840738F09F5F5F4F60
:100B9000220F331F441FAA1FA9F333D00E2E3AF0A1
:100BA000E0E830D091505040E695001CCAF729D0BB
:100BB000FE2F27D0660F771F881FBB1F261737070A
:100BC0004807AB07B0E809F0BB0B802DBF01FF273A
:100BD00093585F4F2AF09E3F510568F085C0CFC003
:100BE0005F3FECF3983EDCF3869577956795B79574
:100BF000F7959F5FC9F7880F911D9695879597F98F
:100C00000895E1E0660F771F881FBB1F6217730707
:100C10008407BA0720F0621B730B840BBA0BEE1F1C
:100C200088F7E0950895E89409C097FB3EF4909505
:100C30008095709561957F4F8F4F9F4F9923A9F0B5
:100C4000F92F96E9BB279395F69587957795679544
:100C5000B795F111F8CFFAF4BB0F11F460FF1BC088
:100C60006F5F7F4F8F4F9F4F16C0882311F096E91B
:100C700011C0772321F09EE8872F762F05C06623C9
:100C800071F096E8862F70E060E02AF09A95660F82
:100C9000771F881FDAF7880F9695879597F908953B
:100CA000990F0008550FAA0BE0E8FEEF161617067D
:100CB000E807F907C0F012161306E407F50798F0E5
:100CC000621B730B840B950B39F40A2661F0232BFE
:100CD000242B252B21F408950A2609F4A140A6957A
:100CE0008FEF811D811D089597F99F6780E870E05F
:100CF00060E008959FEF80EC089500240A94161692
:100D0000170618060906089500240A9412161306F9
:100D1000140605060895092E0394000C11F4882387
:100D200052F0BB0F40F4BF2B11F460FF04C06F5FA3
:100D30007F4F8F4F9F4F089557FD9058440F551F79
:100D400059F05F3F71F04795880F97FB991F61F04D
:100D50009F3F79F087950895121613061406551FC4
:100D6000F2CF4695F1DF08C0161617061806991F30
:100D7000F1CF86957105610508940895E894BB2725
:100D800066277727CB0197F908958ADF08F48FEF5C
:100D900008950EF0A6C0AECF6894A6CFD5DFC8F3F5
:100DA0009923D1F3C6F3DF93CF931F930F93FF9251
:100DB000C92FDD2788232AF02197660F771F881F08
:100DC000DAF720E030E040E85FEB9FE3883920F07D
:100DD000803E30F021968F7756DEECE7F0E003C0DE
:100DE00052DEE9EAF0E08BD08B01BE01EC01FB2E74
:100DF0006F5771097595771F880B990B16DF28E1DE
:100E000032E741E35FE316D0AF2D9801AE01FF90CA
:100E10000F911F91CF91DF9147DE7DCF0BD07BCF1C
:100E20006CDF28F071DF18F0952309F05DCF62CFF9
:100E30001124A5CF81DFA0F3959FD1F3950F50E04A
:100E4000551F629FF001729FBB27F00DB11D639F7C
:100E5000AA27F00DB11DAA1F649F6627B00DA11D22
:100E6000661F829F2227B00DA11D621F739FB00DC8
:100E7000A11D621F839FA00D611D221F749F332738
:100E8000A00D611D231F849F600D211D822F762FD1
:100E90006A2F11249F5750408AF0E1F088234AF0CE
:100EA000EE0FFF1FBB1F661F771F881F915050401A
:100EB000A9F79E3F510570F017CF61CF5F3FECF36C
:100EC000983EDCF3869577956795B795F795E79506
:100ED0009F5FC1F7FE2B880F911D9695879597F917
:100EE00008959F3F31F0915020F48795779567954D
:100EF000B795880F911D9695879597F90895DF937B
:100F0000CF931F930F93FF92EF92DF927B018C019F
:100F1000689405C0DA2EEF018DDFFE01E894A591FB
:100F20002591359145915591AEF3EF01BDDDFE015F
:100F30009701A801DA9479F7DF90EF90FF900F9175
:100F40001F91CF91DF910895052E97FB16F4009421
:100F50000FD057FD05D039D007FC02D046F408C0A9
:100F600050954095309521953F4F4F4F5F4F0895D5
:100F700090958095709561957F4F8F4F9F4F089505
:100F800005D0332312F48A1B9B0B10C0A29FB00123
:100F9000B39FC001A39F700D811D1124911DB29FAD
:100FA000700D811D1124911D0895F0DFB7FF089584
:100FB000821B930B0895EADFA59F900DB49F900DBF
:100FC000A49F800D911D11240895A1E21A2EAA1B41
:100FD000BB1BFD010DC0AA1FBB1FEE1FFF1FA217E9
:100FE000B307E407F50720F0A21BB30BE40BF50BE6
:100FF000661F771F881F991F1A9469F7609570956F
:10100000809590959B01AC01BD01CF010895F894A6
:02101000FFCF10
:1010120000010203040506080755D0A4420000DCC3
:1010220042FED412437DFF434327F1764362D0A4AC
:10103200430001020304051010F800000000101024
:1010420010404000000000100004050607050403DC
:10105200020100000102030102030000000000017E
:101062000101010101020202020000000010204001
:0F10720080201008040201010204080204080192
:00000001FF
